:020000040000FA
:1000000045EF02F0F76A140FF66E000EF7220900B2
:10001000F55012000A0D303433202D204F53524139
:100020004D204F4C454420647269766572200A0D5C
:100030000A0D0000F76A440FF66E000EF722090061
:10004000F55012004F5352414D204F4C454420393A
:10005000367836340000F76A660FF66E000EF72227
:100060000900F550120020207465636864657369A7
:10007000676E2E6265200000F76A880FF66E000E2C
:10008000F7220900F5501200566572746963616CBD
:10009000207363726F6C6C200000F76AAA0FF66E13
:1000A000000EF7220900F5501200526967687420AB
:1000B0007363726F6C6C0000F76AC80FF66E000E07
:1000C000F7220900F5501200496E76657274656476
:1000D00020646973706C61790000F76AEA0FF66E4C
:1000E000000EF7220900F5501200436F6E74726122
:1000F000737420636F6E74726F6C0000F76A0C0F7C
:10010000F66E010EF7220900F55012004561737971
:1001100020696E7465726661636520200000F76A6D
:100120002E0FF66E010EF7220900F550120031363F
:1001300020636861722078203820726F7773000026
:10014000010EEA6EF40EE96EEF500DE0060E016E40
:10015000006A002EFED7012EFBD77B0E006E002E0C
:10016000FED7EF2EF3D7000C080E0201026F0253E8
:100170000CE083960151800B02E1839401D08384CB
:100180008386D89001370207F2D70001000C839ACA
:100190008392FBC101F2E8DF838A000C838A8386A5
:1001A00083980A0E0101F46F0001CADF8388010EF3
:1001B0000101F46F0001C4DF040E0101FB6F0001B7
:1001C000E6DF120E0101FB6F0001E1DF400E0101CD
:1001D000FB6F0001DCDF810E0101FB6F0001D7DF47
:1001E0003F0E0101FB6F0001D2DFA10E0101FB6F89
:1001F0000001CDDFA40E0101FB6F0001C8DFA60ED8
:100200000101FB6F0001C3DFA80E0101FB6F0001BC
:10021000BEDF3F0E0101FB6F0001B9DFAD0E010132
:10022000FB6F0001B4DF8B0E0101FB6F0001AFDF3C
:10023000AF0E0101FB6F0001AADFD30E0101FB6FBE
:100240000001A5DF0101FB6B0001A1DFD50E01015B
:10025000FB6F00019CDF210E0101FB6F000197DFA6
:10026000D80E0101FB6F000192DF0101FB6B000161
:100270008EDFDA0E0101FB6F000189DF120E010132
:10028000FB6F000184DFDB0E0101FB6F00017FDFEC
:10029000350E0101FB6F00017ADFD90E0101FB6F02
:1002A000000175DF220E0101FB6F000170DF2E0ED1
:1002B0000101FB6F00016BDFBAEF05F0240E0101B5
:1002C000F627F6510F0BF96FF639006E0F0E001678
:1002D00000500F0B1009F86FF9C1FBF1000157DF57
:1002E000F8C1FBF154DF0101F751070BB009FA6FB8
:1002F000FB6F00014CDF000C839A838200C201F285
:1003000033DF8392E30E0201016F00012DDF838A48
:10031000000C0101F1511F0801E338D0F1517F08B1
:1003200001E234D0F06BF05104082BE3F1514F0897
:1003300010E3F151E00F050DF3CFF2F1F051F2258A
:10034000036A100FE96E000E0320EA6EEFCFF3F19F
:1003500011D0F1514F080EE2F151B00F050DF3CF5E
:10036000F2F1F051F225036AE96E010E0324EA6E00
:10037000EFCFF3F1F3C100F20001BEDF0101F02B7A
:10038000D2D70201006B0001B7DF01010001CCEF01
:1003900001F0FEC1F1F1BDD7000C0101F56BF55183
:1003A000080811E0F66BF5C1F7F1000187DF180EC0
:1003B0000101F66F200EFE6F0001EBDF0101F62F49
:1003C000F9D7F52BECD70001BBEF05F0EACFFDF133
:1003D000E9CFFCF10101F639F009F86FF827E20FD7
:1003E000F96F320FFB6FF6510F0BF927F927FB2737
:1003F000E90FFA6FFA27FA27F5390F0BFA27FB27CF
:10040000FA37FB37FB1FFB37F5510F0BFB27F8378C
:10041000070EF76F0A0EFA07FB27FDE3F907FA2725
:10042000FDE3F807F927FDE3F707F827FDE3010EE1
:10043000EA6EF70EE96E070EFC15FC9DE926FB0E31
:10044000E95CD8B4FC8DEF50006E08E1FCBD06D02D
:10045000FCB915D0FCB702D0200E03D0FC87FC9964
:10046000300E0026EACFF6F1E9CFF5F100C0FEF13B
:1004700000018FDFF6C1EAFFF5C1E9FF0101EE508F
:10048000FCADDDD700015BEF06F0F86AD09EFE0EF2
:10049000006E060E016E020EE96E000EEA6EEE6A46
:1004A000002EFDD7012EFBD7EA6AE96A400EAF6E37
:1004B000A60EAC6E900EAB6EC180C182C184C19697
:1004C000056A066A106A116A126A136A146A156A62
:1004D000166A5F0E176E186A196A1A6A070E1B6E83
:1004E0001C6A1D6E1E6A140E1F6E7F0E206E140E87
:1004F000216E7F0E226E140E236E240E246E2A0EA1
:10050000256E7F0E266E2A0E276E120E286E230E83
:10051000296E130E2A6E080E2B6E640E2C6E620E60
:100520002D6E360E2E6E490E2F6E550E306E220E2B
:10053000316E500E326E336A050E346E030E356E18
:10054000366A376A386A1C0E396E220E3A6E410ED0
:100550003B6E3C6A3D6A3E6E220E3F6E1C0E406E44
:10056000416A140E426E080E436E3E0E446E080E33
:10057000456E140E466E080E476E486E3E0E496E6E
:10058000080E4A6E4B6E4C6A500E4D6E300E4E6E1B
:100590004F6A506A080E516E526E536E546E556E0D
:1005A000566A600E576E586E596A5A6A200E5B6E14
:1005B000100E5C6E080E5D6E040E5E6E020E5F6EB7
:1005C0003E0E606E510E616E490E626E450E636E98
:1005D0003E0E646E656A420E666E7F0E676E400E5A
:1005E000686E696A420E6A6E610E6B6E510E6C6EB9
:1005F000490E6D6E460E6E6E210E6F6E410E706E60
:10060000450E716E4B0E726E310E736E180E746E57
:10061000140E756E120E766E7F0E776E100E786E5B
:10062000270E796E450E7A6E7B6E7C6E390E7D6E6E
:100630003C0E7E6E4A0E7F6E490E806F816F300ECB
:10064000826F010E836F710E846F090E856F050E28
:10065000866F030E876F360E886F490E896F8A6F1B
:100660008B6F360E8C6F060E8D6F490E8E6F8F6FEF
:10067000290E906F1E0E916F926B360E936F946FD2
:10068000956B966B976B560E986F360E996F9A6BAB
:100690009B6B080E9C6F140E9D6F220E9E6F410E79
:1006A0009F6FA06B140EA16FA26FA36FA46FA56FB5
:1006B000A66B410EA76F220EA86F140EA96F080E2D
:1006C000AA6F020EAB6F010EAC6F510EAD6F090E2B
:1006D000AE6F060EAF6F320EB06F490EB16F790E6E
:1006E000B26F410EB36F3E0EB46F7E0EB56F110E3A
:1006F000B66FB76FB86F7E0EB96F7F0EBA6F490EC7
:10070000BB6FBC6FBD6F360EBE6F3E0EBF6F410E2E
:10071000C06FC16FC26F220EC36F7F0EC46F410ED8
:10072000C56FC66F220EC76F1C0EC86F7F0EC96FD4
:10073000490ECA6FCB6FCC6F410ECD6F7F0ECE6F5F
:10074000090ECF6FD06FD16F010ED26F3E0ED36FF7
:10075000410ED46F490ED56FD66F7A0ED76F7F0ECC
:10076000D86F080ED96FDA6FDB6F7F0EDC6FDD6B31
:10077000410EDE6F7F0EDF6F410EE06FE16B200EEA
:10078000E26F400EE36F410EE46F3F0EE56F010E26
:10079000E66F7F0EE76F080EE86F140EE96F220E0A
:1007A000EA6F410EEB6F7F0EEC6F400EED6FEE6F58
:1007B000EF6FF06F7F0EF16F020EF26F0C0EF36FA2
:1007C000020EF46F7F0EF56FF66F040EF76F080ED2
:1007D000F86F100EF96F7F0EFA6F3E0EFB6F410E31
:1007E000FC6FFD6FFE6F3E0EFF6F7F0E0101006F0D
:1007F000090E016F026F036F060E046F3E0E056F48
:10080000410E066F510E076F210E086F5E0E096FC5
:100810007F0E0A6F090E0B6F190E0C6F290E0D6FEC
:10082000460E0E6F0F6F490E106F116F126F310E63
:10083000136F010E146F156F7F0E166F010E176F79
:10084000186F3F0E196F400E1A6F1B6F1C6F3F0E13
:100850001D6F1F0E1E6F200E1F6F400E206F200E8B
:10086000216F1F0E226F3F0E236F400E246F380E34
:10087000256F400E266F3F0E276F630E286F140EF4
:10088000296F080E2A6F140E2B6F630E2C6F070E44
:100890002D6F080E2E6F700E2F6F080E306F070E23
:1008A000316F610E326F510E336F490E346F450E4A
:1008B000356F430E366F376B7F0E386F410E396FD1
:1008C0003A6F3B6B020E3C6F040E3D6F080E3E6F9D
:1008D000100E3F6F200E406F416B410E426F436F11
:1008E0007F0E446F456B040E466F020E476F010E7C
:1008F000486F020E496F040E4A6F400E4B6F4C6FEB
:100900004D6F4E6F4F6F506B010E516F020E526F55
:10091000040E536F546B200E556F540E566F576F65
:10092000586F780E596F7F0E5A6F480E5B6F440EEA
:100930005C6F5D6F380E5E6F5F6F440E606F616F4E
:10094000626F200E636F380E646F440E656F666FC2
:10095000480E676F7F0E686F380E696F540E6A6FAE
:100960006B6F6C6F180E6D6F080E6E6F7E0E6F6F73
:10097000090E706F010E716F020E726F0C0E736FA5
:10098000520E746F756F766F3E0E776F7F0E786FB5
:10099000080E796F040E7A6F7B6F780E7C6F7D6B1B
:1009A000440E7E6F7D0E7F6F400E806F816B200E38
:1009B000826F400E836F440E846F3D0E856F866B91
:1009C0007F0E876F100E886F280E896F440E8A6F16
:1009D0008B6B8C6B410E8D6F7F0E8E6F400E8F6F09
:1009E000906B7C0E916F040E926F180E936F040E35
:1009F000946F780E956F7C0E966F080E976F040EAD
:100A0000986F996F780E9A6F380E9B6F440E9C6F9B
:100A10009D6F9E6F380E9F6F7C0EA06F140EA16F9E
:100A2000A26FA36F080EA46FA56F140EA66FA76F19
:100A3000180EA86F7C0EA96FAA6F080EAB6F040E7C
:100A4000AC6FAD6F080EAE6F480EAF6F540EB06F47
:100A5000B16FB26F200EB36F040EB46F3F0EB56F5F
:100A6000440EB66F400EB76F200EB86F3C0EB96FD4
:100A7000400EBA6FBB6F200EBC6F7C0EBD6F1C0E9C
:100A8000BE6F200EBF6F400EC06F200EC16F1C0ED8
:100A9000C26F3C0EC36F400EC46F300EC56F400E68
:100AA000C66F3C0EC76F440EC86F280EC96F100E7C
:100AB000CA6F280ECB6F440ECC6F0C0ECD6F500E4C
:100AC000CE6FCF6FD06F3C0ED16F440ED26F640EDD
:100AD000D36F540ED46F4C0ED56F440ED66FD76BB8
:100AE000080ED86F360ED96F410EDA6FDB6BDC6BF8
:100AF000DD6B7F0EDE6FDF6BE06BE16B410EE26F53
:100B0000360EE36F080EE46FE56B100EE66F080E0D
:100B1000E76FE86F100EE96F080EEA6F780EEB6F63
:100B2000460EEC6F410EED6F460EEE6F780EEF6FD6
:100B3000C290C180C182C184C196290E926E020EFC
:100B4000936E900E946EC00E956E968096829684EB
:100B5000F46BF451000102EC00F00101F42B006E83
:100B600000509EA8FED7AD6E1E0EF45DF2E10001AE
:100B7000CEEF00F012D40101F66BF76B00015EECD2
:100B800001F00101F46BF45100011AEC00F00101D5
:100B9000F42B006EFE6F0001C9EC01F0100E010194
:100BA000F45DF1E1F66B020EF76F00015EEC01F00F
:100BB0000101F46BF45100012BEC00F00101F42B66
:100BC000006EFE6F0001C9EC01F0100E0101F45D32
:100BD000F1E1F66B050EF76F00015EEC01F0030E1C
:100BE0000101F46F2D0EFE6F0001C9EC01F001014F
:100BF000F42FF8D7030EF56F2B0EFE6F0001C9EC32
:100C000001F00101F52FF8D7040EF66F2A0EFE6FE2
:100C10000001C9EC01F00101F62FF8D7030EF76FC0
:100C20002B0EFE6F0001C9EC01F00101F72FF8D780
:100C3000030EF86F2D0EFE6F0001C9EC01F00101EB
:100C4000F82FF8D7260EFB6F0001C7EC00F0010E5D
:100C50000101FB6F0001C7EC00F0020E0101FB6F08
:100C60000001C7EC00F0010E0101FB6F0001C7ECB1
:100C700000F0030E0101FB6F0001C7EC00F0300E25
:100C80000101F66F070EF76F00015EEC01F0030E35
:100C90000101F46F300EFE6F0001C9EC01F001019B
:100CA000F42FF8D7080EE96E09C0F6F108C0F5F187
:100CB0000001E6EF01F02F0E0101FB6F0001C7EC10
:100CC00000F0320E0101F46F0001A0EC00F02E0ED6
:100CD0000101FB6F0001C7EC00F00A5064081BE142
:100CE0000B5219E1400E076E07507F080CE007C059
:100CF000FBF1C7EC00F00A0E0101F46F0001A0EC5B
:100D000000F0072AF1D70B6A0A6A400E0101FB6F57
:100D10000001C7EC00F00E2C1CD00F521AE10101AB
:100D2000F66B050EF76F00015EEC01F00101F46B4C
:100D3000F45100013CEC00F00101F42B006EFE6F59
:100D40000001C9EC01F0100E0101F45DF1E1AFD03A
:100D500000010E50640826E10F5224E10101F66BF8
:100D6000050EF76F00015EEC01F00101F46BF45128
:100D700000014DEC00F00101F42B006EFE6F00014C
:100D8000C9EC01F00C0E0101F45DF1E1040EF56F08
:100D9000200EFE6F0001C9EC01F00101F52FF8D71C
:100DA00086D000010E50C8081CE10F521AE1010163
:100DB000F66B050EF76F00015EEC01F00101F46BBC
:100DC000F45100015CEC00F00101F42B006EFE6FA9
:100DD0000001C9EC01F0100E0101F45DF1E167D0F2
:100DE00000010E502C081CE10F2C1AD00101F66BEB
:100DF000050EF76F00015EEC01F00101F46BF45198
:100E000000016DEC00F00101F42B006EFE6F00019B
:100E1000C9EC01F0100E0101F45DF1E148D00001D0
:100E20000E5090081CE10F2C1AD00101F66B050E34
:100E3000F76F00015EEC01F00101F46BF451000169
:100E40007EEC00F00101F42B006EFE6F0001C9EC96
:100E500001F0100E0101F45DF1E129D000010E5006
:100E6000F4081CE10F2C1AD00101F66B050EF76F88
:100E700000015EEC01F00101F46BF45100018FEC14
:100E800000F00101F42B006EFE6F0001C9EC01F0CF
:100E9000100E0101F45DF1E10AD000010E50580876
:100EA00005E10F50020802E10F6A0E6A0101082AEB
:100EB000D8B4092A0A2AD8B40B2A0C2AD8B40D2A85
:0C0EC0000E2AD8B40F2A0001DAD6030075
:020000040030CA
:0E00000000220C0E000180000FC00FE00F4028
:00000001FF
